:0200000480007A
:100000006F004005732F2034930F8000630AFF03B5
:10001000930F90006306FF03930FB0006302FF038A
:10002000170F0000130F4F3F63040F0067000F000E
:10003000732F203463540F006F00400093E19153FD
:10004000171F000023203FFC171F0000232E0FFA6C
:100050006FF01FFF930000001301000093010000E8
:10006000130200009302000013030000930300003A
:100070001304000093040000130500009305000022
:10008000130600009306000013070000930700000A
:1000900013080000930800001309000093090000F2
:1000A000130A0000930A0000130B0000930B0000DA
:1000B000130C0000930C0000130D0000930D0000C2
:1000C000130E0000930E0000130F0000930F0000AA
:1000D000732540F16310050097020000938202012E
:1000E000739052307350447497020000938202015F
:1000F00073905230735000189702000093824202AE
:10010000739052309B021000939252039382F2FF3D
:100110007390023B9302F0017390023A73504030A7
:100120009702000093824201739052307350203046
:100130007350303093010000970200009382C2ECAC
:1001400073905230130510001315F501635C050020
:100150000F00F00F930110009308D0051305000065
:100160007300000093020000638A02007390521033
:10017000B7B200009B82921073902230735000300F
:10018000372500001B05058073200530970200000D
:100190009382420173901234732540F17300203032
:1001A000B72200009B82028073B0023073230030BC
:1001B000B3F26200639402029301200173250030C0
:1001C0009B053000939505023375B5009B03100025
:1001D00093931302631875206F000002930130019E
:1001E000732500309B053000939505023375B500EB
:1001F000930300006318751E9301400173100034CF
:100200007325003493030000631E751C9301500195
:100210007355003473D50734930300006314751CC1
:100220009301600173600834732500349303F00177
:10023000631A751A73D001349301200073250034BA
:10024000930330006310751A93013000F3F5003406
:10025000930330006398751893014000736602346D
:10026000930320006310761893015000F356013475
:100270009303600063987616930160003725AD0BF9
:100280001B05A5DEF315053493032000639C75144C
:1002900093017000372500001B05A5DEF3350534FA
:1002A000B723AD0B9B83A3DE639E75129301800081
:1002B00037C500001B05F5EEF3250534B703AD0B7C
:1002C00063927512930190003725AD0B1B05A5DED7
:1002D00073150534B7C3AD0B9B83F3EE6314751030
:1002E0009301A000372500001B05A5DE73350534FA
:1002F000B723AD0B9B83A3DE6316750E9301B0008D
:1003000037C500001B05F5EE73250534B703AD0BAB
:10031000631A750C9301C00073250034B7C3AD0B8D
:100320009B83F3EE6310750C732510301375050273
:1003300063080502B765000073A00530530000F0A4
:1003400073B00530972500009385C5CB9301D0008D
:1003500027A0050003A5050093031000631475088A
:1003600073251030135545011375150063000506FC
:1003700073D06030732510301355250113751500A7
:100380006304050073D06010B72200009B820280D6
:1003900073B002309702000093820201739012340E
:1003A000730020309301E0001305F00F731500C0B7
:1003B0009303F00F631875029301F0001305F00F1B
:1003C000732500309303F00F631E75000F00F00FCC
:1003D000930110009308D00513050000730000007E
:1003E000631030020F00F00F638001009391110041
:1003F00093E111009308D0051385010073000000FC
:100400000F00F00F930110009308D00513050000B2
:10041000730000009302D00063E651009302F000E5
:1004200063F23202F322203413038000E39C62FA69
:100430000F00F00F930110009308D0051305000082
:1004400073000000F322203413032000E39C62F8C1
:10045000F3221034938242007390123473002030E0
:10046000731000C000000000000000000000000049
:10047000000000000000000000000000000000007C
:1010000000000000000000000000000000000000E0
:1010100000000000000000000000000000000000D0
:1010200000000000000000000000000000000000C0
:1010300000000000000000000000000000000000B0
:081040000000000000000000A8
:1020000001000000000000000000000000000000CF
:040000058000000077
:00000001FF
